:100000000C942A001895000018950000189500001F
:10001000189500001895000018950000189500002C
:10002000189500001895000018950000189500001C
:10003000189500000C947C26189500001895000077
:1000400018950000189500001895000018950000FC
:10005000189500008FE58DBFC0E2E4E94E2E88E0E0
:100060008EBFD8E0F7E05F2EEEEFF7E0A0E6B0E05D
:10007000A89584B7082E877F84BF88E1992781BD22
:1000800091BD88278D933197E9F783E389B980E0A3
:1000900080BD88E18AB96624579A7894D29ADA9812
:1000A0008C988D9A95988E9A96988F9880917A02CE
:1000B000806480937A02E0E0F0E0ADEDB2E09CE095
:1000C0000E946B27A19AA998A69AAE9AD59AD69A19
:1000D000D79AAAEEB2E0EEE3FFE40E9499250E94CF
:1000E000602582E2A9EFB2E08D9388278C930E946D
:1000F000C2080E94CD080E942B090E942B095A9227
:100100004A9280E0A42DB52D8C9381E00E94F624C4
:100110005A924A9280E0A42DB52D8C9381E00E94E2
:10012000F6240E94BE09249682E00E94F2245A928C
:100130004A92A42DB52DECE4FFE40E9499258CE0B1
:100140000E94F6240E946F0A22968CE00E94F224FC
:1001500084E690E00E9484255A924A9280E0A42D81
:10016000B52D8C9381E00E94F6245A924A9281E048
:10017000A42DB52D8C9381E00E94F6240E94BE0927
:10018000249682E00E94F2245A924A92EAEEF2E029
:10019000A42DB52D0E9446278FE00E94F6240E94D0
:1001A0006F0A22968FE00E94F22484E690E00E947B
:1001B00084255A924A9280E0A42DB52D8C9381E03B
:1001C0000E94F6245A924A9283E0A42DB52D8C9376
:1001D00081E00E94F6240E94BE09249682E00E94DB
:1001E000F2245A924A92A42DB52DE8E5FFE40E942C
:1001F00099258FE00E94F6240E946F0A22968FE0D4
:100200000E94F22484E690E00E9484255A924A9249
:1002100080E0A42DB52D8C9381E00E94F6245A92A3
:100220004A9284E0A42DB52D8C9381E00E94F6249F
:100230000E94BE09249682E00E94F2245A924A92B9
:10024000A42DB52DE8E6FFE40E9499258EE00E94DA
:10025000F6240E946F0A22968EE00E94F2245A929F
:100260004A9280E0A42DB52D8C9381E00E94F62463
:100270005A924A9285E0A42DB52D8C9381E00E947C
:10028000F6240E94BE09249682E00E94F2245A922B
:100290004A92A42DB52DE8E5FFE40E9499258FE050
:1002A0000E94F6240E946F0A22968FE00E94F22498
:1002B000E5E0F0E00E944D25DA9A959A0E942B091C
:1002C0005A924A9280E0A42DB52D8C9381E00E9431
:1002D000F6245A924A9282E0A42DB52D8C9381E0A7
:1002E0000E94F6240E94BE09249682E00E94F22415
:1002F0005A924A92A42DB52DE6E7FFE40E94992573
:100300008FE00E94F6240E946F0A22968FE00E94DE
:10031000F22480E0809377025A924A9280E0A42DE2
:10032000B52D8C9381E00E94F6245A924A9283E084
:10033000A42DB52D8C9381E00E94F6240E94BE0965
:10034000249682E00E94F2245A924A92A42DB52D5E
:10035000E6E8FFE40E9499258FE00E94F6240E94BF
:100360006F0A22968FE00E94F2248EE091E00E94B4
:1003700084255A924A9280917702A42DB52D8C93B0
:1003800081E00E94F6245A924A9283E0A42DB52D72
:100390008C9381E00E94F6240E94BE09249682E09C
:1003A0000E94F2245A924A92A42DB52DE6E9FFE468
:1003B0000E94992582E00E94F6240E946F0A2296EC
:1003C00082E00E94F2248EE091E00E9484255A92FD
:1003D0004A9280917702A42DB52D8C9381E00E94E2
:1003E000F6245A924A9283E0A42DB52D8C9381E095
:1003F0000E94F6240E94BE09249682E00E94F22404
:100400005A924A92A42DB52DE8E9FFE40E9499255D
:1004100082E00E94F6240E946F0A229682E00E94E7
:10042000F2248EE091E00E9484255A924A928091B3
:100430007702A42DB52D8C9381E00E94F6245A9268
:100440004A9283E0A42DB52D8C9381E00E94F6247E
:100450000E94BE09249682E00E94F2245A924A9297
:10046000A42DB52DEAE9FFE40E94992582E00E94BF
:10047000F6240E946F0A229682E00E94F2248EE007
:1004800091E00E9484255A924A9280917702A42D8D
:10049000B52D8C9381E00E94F6245A924A9283E013
:1004A000A42DB52D8C9381E00E94F6240E94BE09F4
:1004B000249682E00E94F2245A924A92A42DB52DED
:1004C000ECE9FFE40E94992582E00E94F6240E9454
:1004D0006F0A229682E00E94F2248EE091E00E9450
:1004E0008425A7E7B2E08C918F5F8C93009177020F
:1004F000023011F00C94B9019598DA985A924A9208
:1005000080E0A42DB52D8C9381E00E94F6245A92B0
:100510004A9282E0A42DB52D8C9381E00E94F624AE
:100520000E94BE09249682E00E94F2245A924A92C6
:10053000A42DB52DEEE9FFE40E9499258FE00E94DD
:10054000F6240E946F0A22968FE00E94F2245A92AB
:100550004A9280917702A42DB52D8C9381E00E9460
:10056000F6245A924A9283E0A42DB52D8C9381E013
:100570000E94F6240E94BE09249682E00E94F22482
:100580005A924A92A42DB52DEEEAFFE40E949925D5
:1005900082E00E94F6240E946F0A229682E00E9466
:1005A000F2248EE091E00E9484255A924A92809132
:1005B0007702A42DB52D8C9381E00E94F6245A92E7
:1005C0004A9283E0A42DB52D8C9381E00E94F624FD
:1005D0000E94BE09249682E00E94F2245A924A9216
:1005E000A42DB52DE6E9FFE40E94992582E00E9442
:1005F000F6240E946F0A229682E00E94F2248EE086
:1006000091E00E9484255A924A9280917702A42D0B
:10061000B52D8C9381E00E94F6245A924A9283E091
:10062000A42DB52D8C9381E00E94F6240E94BE0972
:10063000249682E00E94F2245A924A92A42DB52D6B
:10064000E8E9FFE40E94992582E00E94F6240E94D6
:100650006F0A229682E00E94F2248EE091E00E94CE
:1006600084255A924A9280917702A42DB52D8C93BD
:1006700081E00E94F6245A924A9283E0A42DB52D7F
:100680008C9381E00E94F6240E94BE09249682E0A9
:100690000E94F2245A924A92A42DB52DEAE9FFE471
:1006A0000E94992582E00E94F6240E946F0A2296F9
:1006B00082E00E94F2248EE091E00E9484255A920A
:1006C0004A9280917702A42DB52D8C9381E00E94EF
:1006D000F6245A924A9283E0A42DB52D8C9381E0A2
:1006E0000E94F6240E94BE09249682E00E94F22411
:1006F0005A924A92A42DB52DECE9FFE40E94992567
:1007000082E00E94F6240E946F0A229682E00E94F4
:10071000F2248EE091E00E948425A7E7B2E08C915C
:100720008F5F8C9300917702063011F00C94A70232
:100730005A924A9280E0A42DB52D8C9381E00E94BC
:10074000F6245A924A9282E0A42DB52D8C9381E032
:100750000E94F6240E94BE09249682E00E94F224A0
:100760005A924A92A42DB52DE0EBFFE40E94992500
:100770008FE00E94F6240E946F0A22968FE00E946A
:10078000F224E0ECFFE40E943F250E9446255A92A5
:100790004A9280917702A42DB52D8C9381E00E941E
:1007A000F6245A924A9283E0A42DB52D8C9381E0D1
:1007B0000E94F6240E94BE09249682E00E94F22440
:1007C0005A924A92A42DB52DEEEAFFE40E94992593
:1007D00082E00E94F6240E946F0A229682E00E9424
:1007E000F2248EE091E00E948425E0ECFFE40E9478
:1007F0003F250E9446250E94D5155A924A92809123
:100800007702A42DB52D8C9381E00E94F6245A9294
:100810004A9283E0A42DB52D8C9381E00E94F624AA
:100820000E94BE09249682E00E94F2245A924A92C3
:10083000A42DB52DE6E9FFE40E94992582E00E94EF
:10084000F6240E946F0A229682E00E94F2248EE033
:1008500091E00E9484255A924A9280917702A42DB9
:10086000B52D8C9381E00E94F6245A924A9283E03F
:10087000A42DB52D8C9381E00E94F6240E94BE0920
:10088000249682E00E94F2245A924A92A42DB52D19
:10089000E8E9FFE40E94992582E00E94F6240E9484
:1008A0006F0A229682E00E94F2248EE091E00E947C
:1008B00084255A924A9280917702A42DB52D8C936B
:1008C00081E00E94F6245A924A9283E0A42DB52D2D
:1008D0008C9381E00E94F6240E94BE09249682E057
:1008E0000E94F2245A924A92A42DB52DEAE9FFE41F
:1008F0000E94992582E00E94F6240E946F0A2296A7
:1009000082E00E94F2248EE091E00E9484255A92B7
:100910004A9280917702A42DB52D8C9381E00E949C
:10092000F6245A924A9283E0A42DB52D8C9381E04F
:100930000E94F6240E94BE09249682E00E94F224BE
:100940005A924A92A42DB52DECE9FFE40E94992514
:1009500082E00E94F6240E946F0A229682E00E94A2
:10096000F2248EE091E00E948425A7E7B2E08C910A
:100970008F5F8C935A924A9280E0A42DB52D8C9370
:1009800081E00E94F6245A924A9282E0A42DB52D6D
:100990008C9381E00E94F6240E94BE09249682E096
:1009A0000E94F2245A924A92A42DB52DE4ECFFE461
:1009B0000E9499258FE00E94F6240E946F0A2296D9
:1009C0008FE00E94F2245A924A9280917702A42DDD
:1009D000B52D8C9381E00E94F6245A924A9283E0CE
:1009E000A42DB52D8C9381E00E94F6240E94BE09AF
:1009F000249682E00E94F2245A924A92A42DB52DA8
:100A0000EEEAFFE40E94992582E00E94F6240E940B
:100A10006F0A229682E00E94F2248EE091E00E940A
:100A200084255A924A9280917702A42DB52D8C93F9
:100A300081E00E94F6245A924A9283E0A42DB52DBB
:100A40008C9381E00E94F6240E94BE09249682E0E5
:100A50000E94F2245A924A92A42DB52DE6E9FFE4B1
:100A60000E94992582E00E94F6240E946F0A229635
:100A700082E00E94F2248EE091E00E948425E0EC66
:100A8000FFE40E943F250E94462588E290E00E94F4
:100A90008425A2E3B2E0BA93AA930E949715229606
:100AA000A2E3B2E0E4EDFFE40E948B2711F00C9486
:100AB0003F050E94D5155A924A9280917702A42D43
:100AC000B52D8C9381E00E94F6245A924A9283E0DD
:100AD000A42DB52D8C9381E00E94F6240E94BE09BE
:100AE000249682E00E94F2245A924A92A42DB52DB7
:100AF000E8E9FFE40E94992582E00E94F6240E9422
:100B00006F0A229682E00E94F2248EE091E00E9419
:100B100084255A924A9280917702A42DB52D8C9308
:100B200081E00E94F6245A924A9283E0A42DB52DCA
:100B30008C9381E00E94F6240E94BE09249682E0F4
:100B40000E94F2245A924A92A42DB52DEAE9FFE4BC
:100B50000E94992582E00E94F6240E946F0A229644
:100B600082E00E94F2248EE091E00E9484255A9255
:100B70004A9280917702A42DB52D8C9381E00E943A
:100B8000F6245A924A9283E0A42DB52D8C9381E0ED
:100B90000E94F6240E94BE09249682E00E94F2245C
:100BA0005A924A92A42DB52DECE9FFE40E949925B2
:100BB00082E00E94F6240E946F0A229682E00E9440
:100BC000F2248EE091E00E948425A7E7B2E08C91A8
:100BD0008F5F8C935A924A9280E0A42DB52D8C930E
:100BE00081E00E94F6245A924A9282E0A42DB52D0B
:100BF0008C9381E00E94F6240E94BE09249682E034
:100C00000E94F2245A924A92A42DB52DE8EDFFE4F9
:100C10000E9499258FE00E94F6240E946F0A229676
:100C20008FE00E94F224E8EEFFE40E943F2582E27A
:100C30000E944925E2EFFFE40E943F2582E20E94E4
:100C400049250E9446255A924A9280917702A42D06
:100C5000B52D8C9381E00E94F6245A924A9283E04B
:100C6000A42DB52D8C9381E00E94F6240E94BE092C
:100C7000249682E00E94F2245A924A92A42DB52D25
:100C8000EEEAFFE40E94992582E00E94F6240E9489
:100C90006F0A229682E00E94F2248EE091E00E9488
:100CA00084255A924A9280917702A42DB52D8C9377
:100CB00081E00E94F6245A924A9283E0A42DB52D39
:100CC0008C9381E00E94F6240E94BE09249682E063
:100CD0000E94F2245A924A92A42DB52DE6E9FFE42F
:100CE0000E94992582E00E94F6240E946F0A2296B3
:100CF00082E00E94F22488E290E00E948425A2E330
:100D0000B2E0BA93AA930E9497152296A2E3B2E0AA
:100D1000E4EDFFE40E948B2711F00C947B060E9407
:100D2000D5158EE091E00E9484255A924A928091D6
:100D30007702A42DB52D8C9381E00E94F6245A925F
:100D40004A9283E0A42DB52D8C9381E00E94F62475
:100D50000E94BE09249682E00E94F2245A924A928E
:100D6000A42DB52DE8E9FFE40E94992582E00E94B8
:100D7000F6240E946F0A229682E00E94F2248EE0FE
:100D800091E00E9484255A924A9280917702A42D84
:100D9000B52D8C9381E00E94F6245A924A9283E00A
:100DA000A42DB52D8C9381E00E94F6240E94BE09EB
:100DB000249682E00E94F2245A924A92A42DB52DE4
:100DC000EAE9FFE40E94992582E00E94F6240E944D
:100DD0006F0A229682E00E94F2248EE091E00E9447
:100DE00084255A924A9280917702A42DB52D8C9336
:100DF00081E00E94F6245A924A9283E0A42DB52DF8
:100E00008C9381E00E94F6240E94BE09249682E021
:100E10000E94F2245A924A92A42DB52DECE9FFE4E7
:100E20000E94992582E00E94F6240E946F0A229671
:100E300082E00E94F22484E690E00E9484255A9287
:100E40004A9280917702A42DB52D8C9381E00E9467
:100E5000F6245A924A9283E0A42DB52D8C9381E01A
:100E60000E94F6240E94BE09249682E00E94F22489
:100E7000A7E7B2E08C918F5F8C935A924A9280914F
:100E80007702A42DB52D8C9381E00E94F6245A920E
:100E90004A9283E0A42DB52D8C9381E00E94F62424
:100EA0000E94BE09249682E00E94F2245A924A923D
:100EB000A42DB52DEEEAFFE40E94992582E00E9460
:100EC000F6240E946F0A229682E00E94F22482E3B6
:100ED00090E00E9484255A924A9280917702A42D34
:100EE000B52D8C9381E00E94F6245A924A9283E0B9
:100EF000A42DB52D8C9381E00E94F6240E94BE099A
:100F0000249682E00E94F2245A924A92A42DB52D92
:100F1000E6E9FFE40E94992582E00E94F6240E94FF
:100F20006F0A229682E00E94F22482E390E00E94FF
:100F300084255A924A9280917702A42DB52D8C93E4
:100F400081E00E94F6245A924A9283E0A42DB52DA6
:100F50008C9381E00E94F6240E94BE09249682E0D0
:100F60000E94F2245A924A92A42DB52DE8E9FFE49A
:100F70000E94992582E00E94F6240E946F0A229620
:100F800082E00E94F22482E390E00E9484255A923B
:100F90004A9280917702A42DB52D8C9381E00E9416
:100FA000F6245A924A9283E0A42DB52D8C9381E0C9
:100FB0000E94F6240E94BE09249682E00E94F22438
:100FC0005A924A92A42DB52DEAE9FFE40E94992590
:100FD00082E00E94F6240E946F0A229682E00E941C
:100FE000F22482E390E00E9484255A924A928091F2
:100FF0007702A42DB52D8C9381E00E94F6245A929D
:101000004A9283E0A42DB52D8C9381E00E94F624B2
:101010000E94BE09249682E00E94F2245A924A92CB
:10102000A42DB52DECE9FFE40E94992582E00E94F1
:10103000F6240E946F0A229682E00E94F22482E344
:1010400090E00E9484255A924A9280917702A42DC2
:10105000B52D8C9381E00E94F6245A924A9283E047
:10106000A42DB52D8C9381E00E94F6240E94BE0928
:10107000249682E00E94F2245A924A92A42DB52D21
:10108000EAEFFFE40E94992582E00E94F6240E9484
:101090006F0A229682E00E94F22482E390E00E948E
:1010A0008425A7E7B2E08C918F5F8C930091770243
:1010B0000E3011F00C943D0780E0809377020E947F
:1010C0002B095A924A9280E0A42DB52D8C9381E091
:1010D0000E94F6245A924A9282E0A42DB52D8C9358
:1010E00081E00E94F6240E94BE09249682E00E94BC
:1010F000F2245A924A92A42DB52DECEFFFE40E94FF
:1011000099258FE00E94F6240E946F0A22968FE0B4
:101110000E94F2240E94D515DA9AECE0F0E50E94D4
:101120003F250E94462582E390E00E948425E6E167
:10113000F0E50E943F250E944625E3E0F0E00E9492
:101140004D25DA980E94D5150E942B09DA9A0E9443
:1011500016210E94E5150E94C6230E9453170E9483
:10116000A01C0E94201D0E94DF1E0E94F91A0E94EE
:101170007822DA98EAE0F0E00E944D250C94A60867
:10118000F894FFCFDF98EF93FF93E4EEF3E00E9433
:101190005325FF91EF91DF9A0895DE98DD985A92DA
:1011A0004A9281E2A42DB52D8C9381E00E94F62411
:1011B0000E94AC09229681E00E94F2245A924A923F
:1011C00088ECA42DB52D8C9381E00E94F6240E941A
:1011D000AC09229681E00E94F2245A924A9286E05B
:1011E000A42DB52D8C9381E00E94F6240E94AC09B9
:1011F000229681E00E94F2245A924A9283E1A42D21
:10120000B52D8C9381E00E94F6240E94AC092296B1
:1012100081E00E94F2245A924A9280E2A42DB52DD8
:101220008C9381E00E94F6240E94AC09229681E012
:101230000E94F2245A924A928CE0A42DB52D8C93F0
:1012400081E00E94F6240E94AC09229681E00E946F
:10125000F224DE9A089582E00E949325DE98DD98BC
:101260005A924A9280E2A42DB52D8C9381E00E947F
:10127000F6240E94AC09229681E00E94F2245A9240
:101280004A9280E8A42DB52D8C9381E00E94F6242B
:101290000E94AC09229681E00E94F2245A924A925E
:1012A00080E4A42DB52D8C9381E00E94F6240E9449
:1012B000AC09229681E00E94F224DD9A80E090E061
:1012C000A881B9818D939C93A881B9810D911C91BE
:1012D000073F51E0150718F011F00C9485095A9258
:1012E0004A9280E0A42DB52D8C9381E00E94F624D3
:1012F0000E94B509229681E00E94F224A881B9815A
:101300000E94FA2410F40C946409DE9A82E0481AD0
:101310008827580A229608955A924A928DE0A42D61
:10132000B52D8C9381E00E94F6240E94AC09229690
:1013300081E00E94F22408955A924A928CE0A42DF2
:10134000B52D8C9381E00E94F6240E94AC09229670
:1013500081E00E94F2240895DE98DD9891E0A88152
:10136000B9810E945625DE9A0895DE98DD9A91E0B3
:10137000A881B9810E945625DE9A089581E00E94D5
:1013800093255A924A9280E2A42DB52D8C9381E048
:101390000E94F6240E94AC09229681E00E94F22469
:1013A000EF93FF93E4EEF3E00E945325FF91EF915A
:1013B000DE98DD98AC81BD810C9146E0049FA88148
:1013C000B9810C92A881B9818C9180588C9391E05D
:1013D000A881B9810E945625AA81BB810C9140E465
:1013E000040FA881B9810C9391E0A881B9810E9472
:1013F0005625DE9A81E0481A8827580A22960895D1
:1014000082E00E94932581E00E949325DE98DD987A
:101410005A924A9280E2A42DB52D8C9381E00E94CD
:10142000F6240E94AC09229681E00E94F2245A928E
:101430004A9280E8A42DB52D8C9381E00E94F62479
:101440000E94AC09229681E00E94F2245A924A92AC
:1014500080E4A42DB52D8C9381E00E94F6240E9497
:10146000AC09229681E00E94F224DD9A80E090E0AF
:10147000AA81BB818D939C93AA81BB810D911C9104
:10148000073F51E0150718F011F00C94680A0E940C
:10149000EF24A881B9810E949F250C920E94EC2420
:1014A0005A924A92AA81BB818C91A42DB52D8C931E
:1014B00081E00E94F6240E94B509229681E00E94F4
:1014C000F224AA81BB810E94FA2410F40C943C0AF5
:1014D000DE9A83E0481A8827580A2496089581E006
:1014E0000E94932582E00E94932581E00E9493252B
:1014F00081E00E94932581E00E949325AA85BB8507
:101500000E948527A885B9858C9381E0AC81BD8137
:101510008C93A885B9854C91AC81BD810C91041741
:1015200018F011F00C94F012AC81BD818C91EA8519
:10153000FB8501E00A93AF81B8850E944B27AE81FD
:10154000BF81E0E2F0E50E948B2711F00C94AE0A17
:10155000EEE0F7E20E94EC240C94A512E2E2F0E542
:101560000E948B2711F00C94BB0AE4E1F7E20E9481
:10157000EC240C94A512E4E2F0E50E948B2711F014
:101580000C94C80AEAE1F7E20E94EC240C94A5123C
:10159000E6E2F0E50E948B2711F00C94D50AE0E218
:1015A000F7E20E94EC240C94A512E8E2F0E50E9418
:1015B0008B2711F00C94E20AE6E2F7E20E94EC2499
:1015C0000C94A512EAE2F0E50E948B2711F00C942E
:1015D000EF0AECE2F7E20E94EC240C94A512ECE294
:1015E000F0E50E948B2711F00C94FC0AE2E3F7E28D
:1015F0000E94EC240C94A512EEE2F0E50E948B27E9
:1016000011F00C94090BE8E3F7E20E94EC240C942F
:10161000A512E0E3F0E50E948B2711F00C94160B65
:10162000EEE3F7E20E94EC240C94A512E2E3F0E56D
:101630000E948B2711F00C94230BE4E4F7E20E9444
:10164000EC240C94A512E4E3F0E50E948B2711F042
:101650000C94300BEAE4F7E20E94EC240C94A512FF
:10166000E6E3F0E50E948B2711F00C943D0BE0E5DA
:10167000F7E20E94EC240C94A512E8E3F0E50E9446
:101680008B2711F00C944A0BE6E5F7E20E94EC245C
:101690000C94A512EAE3F0E50E948B2711F00C945C
:1016A000570BECE5F7E20E94EC240C94A512ECE356
:1016B000F0E50E948B2711F00C94640BE2E6F7E250
:1016C0000E94EC240C94A512EEE3F0E50E948B2717
:1016D00011F00C94710BE8E6F7E20E94EC240C94F4
:1016E000A512E0E4F0E50E948B2711F00C947E0B2C
:1016F000EEE6F7E20E94EC240C94A512E2E4F0E599
:101700000E948B2711F00C948B0BE4E7F7E20E9408
:10171000EC240C94A512E4E4F0E50E948B2711F070
:101720000C94980BEAE7F7E20E94EC240C94A512C3
:10173000E6E4F0E50E948B2711F00C94A50BE0E89D
:10174000F7E20E94EC240C94A512E8E4F0E50E9474
:101750008B2711F00C94B20BE6E8F7E20E94EC2420
:101760000C94A512EAE4F0E50E948B2711F00C948A
:10177000BF0BECE8F7E20E94EC240C94A512ECE419
:10178000F0E50E948B2711F00C94CC0BE2E9F7E214
:101790000E94EC240C94A512EEE4F0E50E948B2745
:1017A00011F00C94D90BE8E9F7E20E94EC240C94B8
:1017B000A512E0E5F0E50E948B2711F00C94E60BF2
:1017C000EEE9F7E20E94EC240C94A512E2E5F0E5C4
:1017D0000E948B2711F00C94F30BE4EAF7E20E94CD
:1017E000EC240C94A512E4E5F0E50E948B2711F09F
:1017F0000C94000CEAEAF7E20E94EC240C94A51287
:10180000E6E5F0E50E948B2711F00C940D0CE0EB5F
:10181000F7E20E94EC240C94A512E8E5F0E50E94A2
:101820008B2711F00C941A0CE6EBF7E20E94EC24E3
:101830000C94A512EAE5F0E50E948B2711F00C94B8
:10184000270CECEBF7E20E94EC240C94A512ECE5DB
:10185000F0E50E948B2711F00C94340CE2ECF7E2D7
:101860000E94EC240C94A512EEE5F0E50E948B2773
:1018700011F00C94410CE8ECF7E20E94EC240C947B
:10188000A512E0E6F0E50E948B2711F00C944E0CB7
:10189000EEECF7E20E94EC240C94A512E2E6F0E5EF
:1018A0000E948B2711F00C945B0CE4EDF7E20E9490
:1018B000EC240C94A512E4E6F0E50E948B2711F0CD
:1018C0000C94680CEAEDF7E20E94EC240C94A5124B
:1018D000E6E6F0E50E948B2711F00C94750CE0EE23
:1018E000F7E20E94EC240C94A512E8E6F0E50E94D1
:1018F0008B2711F00C94820CE6EEF7E20E94EC24A8
:101900000C94A512EAE6F0E50E948B2711F00C94E6
:101910008F0CECEEF7E20E94EC240C94A512ECE69E
:10192000F0E50E948B2711F00C949C0CE2EFF7E29B
:101930000E94EC240C94A512EEE6F0E50E948B27A1
:1019400011F00C94A90CE8EFF7E20E94EC240C943F
:10195000A512E0E7F0E50E948B2711F00C94B60C7D
:10196000EEEFF7E20E94EC240C94A512E2E7F0E51A
:101970000E948B2711F00C94C30CE4E0F8E20E9463
:10198000EC240C94A512E4E7F0E50E948B2711F0FB
:101990000C94D00CEAE0F8E20E94EC240C94A5121E
:1019A000E6E7F0E50E948B2711F00C94DD0CE0E1F6
:1019B000F8E20E94EC240C94A512E8E7F0E50E94FE
:1019C0008B2711F00C94EA0CE6E1F8E20E94EC247B
:1019D0000C94A512EAE7F0E50E948B2711F00C9415
:1019E000F70CECE1F8E20E94EC240C94A512ECE771
:1019F000F0E50E948B2711F00C94040DE2E2F8E26E
:101A00000E94EC240C94A512EEE7F0E50E948B27CF
:101A100011F00C94110DE8E2F8E20E94EC240C9411
:101A2000A512E0E8F0E50E948B2711F00C941E0D42
:101A3000EEE2F8E20E94EC240C94A512E2E8F0E554
:101A40000E948B2711F00C942B0DE4E3F8E20E9426
:101A5000EC240C94A512E4E8F0E50E948B2711F029
:101A60000C94380DEAE3F8E20E94EC240C94A512E1
:101A7000E6E8F0E50E948B2711F00C94450DE0E4B8
:101A8000F8E20E94EC240C94A512E8E8F0E50E942C
:101A90008B2711F00C94520DE6E4F8E20E94EC243E
:101AA0000C94A512EAE8F0E50E948B2711F00C9443
:101AB0005F0DECE4F8E20E94EC240C94A512ECE833
:101AC000F0E50E948B2711F00C946C0DE2E5F8E232
:101AD0000E94EC240C94A512EEE8F0E50E948B27FE
:101AE00011F00C94790DE8E5F8E20E94EC240C94D6
:101AF000A512E0E9F0E50E948B2711F00C94860D09
:101B0000EEE5F8E20E94EC240C94A512E2E9F0E57F
:101B10000E948B2711F00C94930DE4E6F8E20E94EA
:101B2000EC240C94A512E4E9F0E50E948B2711F057
:101B30000C94A00DEAE6F8E20E94EC240C94A512A5
:101B4000E6E9F0E50E948B2711F00C94AD0DE0E77B
:101B5000F8E20E94EC240C94A512E8E9F0E50E945A
:101B60008B2711F00C94BA0DE6E7F8E20E94EC2402
:101B70000C94A512EAE9F0E50E948B2711F00C9471
:101B8000C70DECE7F8E20E94EC240C94A512ECE9F6
:101B9000F0E50E948B2711F00C94D40DEAE4F7E2F3
:101BA0000E94EC240C94A512EEE9F0E50E948B272C
:101BB00011F00C94E10DE6EEF7E20E94EC240C9497
:101BC000A512E0EAF0E50E948B2711F00C94EE0DCF
:101BD000EEEEF5E20E94EC240C94A512E2EAF0E5A8
:101BE0000E948B2711F00C94FB0DE4EFF5E20E94AC
:101BF000EC240C94A512E4EAF0E50E948B2711F086
:101C00000C94080EEAEFF5E20E94EC240C94A51265
:101C1000E6EAF0E50E948B2711F00C94150EE0E047
:101C2000F6E20E94EC240C94A512E8EAF0E50E948A
:101C30008B2711F00C94220EE6E0F6E20E94EC24D1
:101C40000C94A512EAEAF0E50E948B2711F00C949F
:101C50002F0EECE0F6E20E94EC240C94A512ECEAC4
:101C6000F0E50E948B2711F00C943C0EE2E1F6E2C5
:101C70000E94EC240C94A512EEEAF0E50E948B275A
:101C800011F00C94490EE8E1F6E20E94EC240C9469
:101C9000A512E0EBF0E50E948B2711F00C94560E94
:101CA000E2E6F7E20E94EC240C94A512E2EBF0E5E8
:101CB0000E948B2711F00C94630EEEEFF7E20E9466
:101CC000EC240C94A512E4EBF0E50E948B2711F0B4
:101CD0000C94700EEEE1F6E20E94EC240C94A51236
:101CE000E6EBF0E50E948B2711F00C947D0EE4E208
:101CF000F6E20E94EC240C94A512E8EBF0E50E94B9
:101D00008B2711F00C948A0EEAE2F6E20E94EC2492
:101D10000C94A512EAEBF0E50E948B2711F00C94CD
:101D2000970EE0E3F6E20E94EC240C94A512ECEB93
:101D3000F0E50E948B2711F00C94A40EE6E3F6E286
:101D40000E94EC240C94A512EEEBF0E50E948B2788
:101D500011F00C94B10EECE3F6E20E94EC240C942A
:101D6000A512E0ECF0E50E948B2711F00C94BE0E5A
:101D7000E2E4F6E20E94EC240C94A512E2ECF0E519
:101D80000E948B2711F00C94CB0EE8E4F6E20E943F
:101D9000EC240C94A512EAEFFFE40E948B2711F0CB
:101DA0000C94D80EEEE4F6E20E94EC240C94A512FA
:101DB000E4ECF0E50E948B2711F00C94E50EE4E5CD
:101DC000F6E20E94EC240C94A512E6ECF0E50E94E9
:101DD0008B2711F00C94F20EE6E8F7E20E94EC2457
:101DE0000C94A512E8ECF0E50E948B2711F00C94FE
:101DF000FF0EEAE5F6E20E94EC240C94A512EAEC50
:101E0000F0E50E948B2711F00C940C0FE0E6F6E24F
:101E10000E94EC240C94A512ECECF0E50E948B27B8
:101E200011F00C94190FE6E6F6E20E94EC240C94F3
:101E3000A512EEECF0E50E948B2711F00C94260F12
:101E4000E2E9F7E20E94EC240C94A512E0EDF0E543
:101E50000E948B2711F00C94330FECE6F6E20E94FF
:101E6000EC240C94A512E2EDF0E50E948B2711F012
:101E70000C94400FE4E7F7E20E94EC240C94A512C6
:101E8000E4EDF0E50E948B2711F00C944D0FE2E792
:101E9000F6E20E94EC240C94A512E6EDF0E50E9417
:101EA0008B2711F00C945A0FEEE9F7E20E94EC2414
:101EB0000C94A512E8EDF0E50E948B2711F00C942C
:101EC000670FEAE3F8E20E94EC240C94A512EAED15
:101ED000F0E50E948B2711F00C94740FE8E7F6E20E
:101EE0000E94EC240C94A512ECEDF0E50E948B27E7
:101EF00011F00C94810FEEE7F6E20E94EC240C94B2
:101F0000A512EEEDF0E50E948B2711F00C948E0FD8
:101F1000E4EAF7E20E94EC240C94A512E0EEF0E56E
:101F20000E948B2711F00C949B0FE0E4F8E20E94D2
:101F3000EC240C94A512E2EEF0E50E948B2711F040
:101F40000C94A80FE6E5F7E20E94EC240C94A5128D
:101F5000E4EEF0E50E948B2711F00C94B50FE2EF50
:101F6000F7E20E94EC240C94A512E6EEF0E50E9444
:101F70008B2711F00C94C20FECEBF7E20E94EC24DB
:101F80000C94A512E8EEF0E50E948B2711F00C945A
:101F9000CF0FE4E8F6E20E94EC240C94A512EAEEDE
:101FA000F0E50E948B2711F00C94DC0FEAE8F6E2D2
:101FB0000E94EC240C94A512ECEEF0E50E948B2715
:101FC00011F00C94E90FE6E7F8E20E94EC240C947F
:101FD000A512EEEEF0E50E948B2711F00C94F60F9F
:101FE000E4EDF7E20E94EC240C94A512E0EFF0E59A
:101FF0000E948B2711F00C940310E0E7F8E20E9496
:10200000EC240C94A512ECE9FFE40E948B2711F05C
:102010000C941010E0E9F6E20E94EC240C94A51256
:10202000E2EFF0E50E948B2711F00C941D10E6E919
:10203000F6E20E94EC240C94A512EAE9FFE40E9467
:102040008B2711F00C942A10E8EAF6E20E94EC24A7
:102050000C94A512E4EFF0E50E948B2711F00C948C
:102060003710EEEAF6E20E94EC240C94A512E6EF9B
:10207000F0E50E948B2711F00C944410ECE9F6E295
:102080000E94EC240C94A512E8EFF0E50E948B2747
:1020900011F00C945110E2EAF6E20E94EC240C9448
:1020A000A512E8E9FFE40E948B2711F00C945E1062
:1020B000E4EBF6E20E94EC240C94A512EAEFF0E5C2
:1020C0000E948B2711F00C946B10EAEBF6E20E9451
:1020D000EC240C94A512E6E9FFE40E948B2711F092
:1020E0000C947810E0ECF6E20E94EC240C94A5121B
:1020F000ECEFF0E50E948B2711F00C948510E6ECD4
:10210000F6E20E94EC240C94A512EEEFF0E50E949A
:102110008B2711F00C949210ECEEF7E20E94EC2465
:102120000C94A512E0E0F1E50E948B2711F00C94CD
:102130009F10ECECF6E20E94EC240C94A512EEEA5F
:10214000FFE40E948B2711F00C94AC10E2EDF6E254
:102150000E94EC240C94A512E2E0F1E50E948B278A
:1021600011F00C94B910E8EDF6E20E94EC240C9406
:10217000A512E4E0F1E50E948B2711F00C94C61043
:10218000EEEDF6E20E94EC240C94A512E6E0F1E5F7
:102190000E948B2711F00C94D310E4EEF6E20E941B
:1021A000EC240C94A512E8E0F1E50E948B2711F0D5
:1021B0000C94E010EAEEF6E20E94EC240C94A512D6
:1021C000EAE0F1E50E948B2711F00C94ED10E0EFAE
:1021D000F6E20E94EC240C94A512ECE0F1E50E94DA
:1021E0008B2711F00C94FA10E6EFF6E20E94EC2433
:1021F0000C94A512EEE0F1E50E948B2711F00C94EF
:102200000711ECEFF6E20E94EC240C94A512E0E139
:10221000F1E50E948B2711F00C941411E2E0F7E233
:102220000E94EC240C94A512E2E1F1E50E948B27B8
:1022300011F00C942111E8E0F7E20E94EC240C94D8
:10224000A512E4E1F1E50E948B2711F00C942E1108
:10225000E2E8F8E20E94EC240C94A512E6E1F1E534
:102260000E948B2711F00C943B11EEE8F8E20E94DB
:10227000EC240C94A512E8E1F1E50E948B2711F003
:102280000C944811E8E8F8E20E94EC240C94A512A2
:10229000EAE1F1E50E948B2711F00C945511E4E975
:1022A000F8E20E94EC240C94A512ECE1F1E50E9406
:1022B0008B2711F00C946211EAECF8E20E94EC24F6
:1022C0000C94A512EEE1F1E50E948B2711F00C941D
:1022D0006F11EAE9F8E20E94EC240C94A512E0E206
:1022E000F1E50E948B2711F00C947C11ECEDF8E2E3
:1022F0000E94EC240C94A512E2E2F1E50E948B27E7
:1023000011F00C948911E0E0F9E20E94EC240C94A5
:10231000A512E4E2F1E50E948B2711F00C949611CE
:10232000E6E0F9E20E94EC240C94A512E6E2F1E565
:102330000E948B2711F00C94A311E4ECF8E20E94A8
:10234000EC240C94A512E8E2F1E50E948B2711F031
:102350000C94B011E8E1F9E20E94EC240C94A5126F
:10236000EAE2F1E50E948B2711F00C94BD11E4E242
:10237000F9E20E94EC240C94A512ECE2F1E50E9433
:102380008B2711F00C94CA11E4EFF8E20E94EC24C0
:102390000C94A512EEE2F1E50E948B2711F00C944B
:1023A000D711E0EDF8E20E94EC240C94A512E0E3D2
:1023B000F1E50E948B2711F00C94E411E2EEF8E2B3
:1023C0000E94EC240C94A512E2E3F1E50E948B2715
:1023D00011F00C94F111ECEAF8E20E94EC240C9458
:1023E000A512E4E3F1E50E948B2711F00C94FE1195
:1023F000EEEEF8E20E94EC240C94A512E6E3F1E57F
:102400000E948B2711F00C940B12ECE0F9E20E9471
:10241000EC240C94A512E8E3F1E50E948B2711F05F
:102420000C941812E0EAF8E20E94EC240C94A51235
:10243000EAE3F1E50E948B2711F00C942512EAEFF4
:10244000F8E20E94EC240C94A512ECE3F1E50E9462
:102450008B2711F00C943212EEE1F9E20E94EC2489
:102460000C94A512EEE3F1E50E948B2711F00C9479
:102470003F12E2EBF8E20E94EC240C94A512E0E497
:10248000F1E50E948B2711F00C944C12E6EDF8E276
:102490000E94EC240C94A512E9EFF2E00E948D2733
:1024A00011F00C945912E8EEF8E20E94EC240C941E
:1024B000A512E2E4F1E50E948B2711F00C9466125C
:1024C000E2E1F9E20E94EC240C94A512E4E4F1E5C7
:1024D0000E948B2711F00C947312E6EAF8E20E9436
:1024E000EC240C94A512E6E4F1E50E948B2711F090
:1024F0000C948012EEEBF8E20E94EC240C94A512EE
:10250000E8E4F1E50E948B2711F00C948D12EAE2C9
:10251000F9E20E94EC240C94A512EAE4F1E50E9491
:102520008B2711F00C949A12E0E3F9E20E94EC245C
:102530000C94A512ECE4F1E50E948B2711F00C94A9
:10254000A512E8EBF8E20E94EC2481E0AA81BB81AD
:102550008C93AA81BB810C91053018F011F00C947A
:10256000D3120E94EF24A881B9810E949F250C926A
:102570000E94EC245A924A92AA81BB818C91A42D8C
:10258000B52D8C9381E00E94F6240E94B509229615
:1025900081E00E94F224AA81BB818C918F5F8C9391
:1025A00010F40C94A91280E0A881B9818C935A92FE
:1025B0004A92AA81BB818C91A42DB52D8C9381E088
:1025C0000E94F6240E94B509229681E00E94F2241E
:1025D000AC81BD818C918F5F8C9310F40C94890A2F
:1025E000DE9A86E0481A8827580A2A9608957F4975
:1025F000494931007C4A4A4931007F4949493600FE
:102600007C54542800007F01010103007C04040471
:102610000C00E0514F41FF00E0544C44FC007C555D
:102620005455440038555455180077087F087700F2
:102630006C107C106C004149494936004454545494
:1026400028007F1008047F007C2010087C007F7F1A
:102650007F7F7F007842241278007C10284400009D
:1026600020413F017F0020443C047C007C0810088E
:102670007C007C1010107C007F0101017F007C0435
:1026800004047C0004047C040400472810080700AC
:102690007F7F7F7F7F000C1010107C000C127F1258
:1026A0000C0018247E2418007F7F7F7F41007C402F
:1026B0004040FC007F7F7F4141007C4078407C00AF
:1026C0007F7F414141007C407840FC007C5050209D
:1026D00000007F41414141004141414141004141B0
:1026E00041417F007C5020007C00224149493E004E
:1026F0002844545438007F083E413E007C10384442
:102700003800462919097F00085434147C003E51D2
:1027100049453E0000427F40000042615149460069
:102720002241494936001814127F100027454545BB
:1027300039003E4949493200611109050300364913
:1027400049493600264949493E007E0909097E006B
:102750007F49494936003E41414122007F41414184
:102760003E007F49494941007F09090901003E4176
:1027700049493A007F0808087F0000417F41000076
:10278000204141413F007F08142241007F404040EA
:1027900040007F0204027F007F0408107F003E415A
:1027A00041413E007F09090906003E4151617E001A
:1027B0007F091929460006494949300001017F0176
:1027C00001003F4040403F001F2040201F007F206D
:1027D00010207F00631408146300030478040300CE
:1027E0006151494543002054545478007F48444483
:1027F0003800384444442800384444487F00385462
:102800005454180000047E0500000C52524A3C004B
:102810007F080404780000447D4000000040443DEF
:1028200000007F201028440000417F4000007C040D
:1028300018047C007C0804047800384444443800C0
:102840007C1424241800182424147C007C0404081C
:102850000000085454542000043F444000003C4011
:1028600040407C001C2040201C003C4030403C008C
:102870004428102844000C5050483C004464544CF8
:102880004400000000000000006060000000080834
:102890000808080000363600000000060909060096
:1028A000007F414100000041417F0000552A552A28
:1028B000550007097F09070040404040400000568E
:1028C00036000000404000707000404000000000F2
:1028D0001414141414000201510906007C7C000039
:1028E000000000005F000000000700070000147FE8
:1028F000147F1400221408142200231308646200B9
:102900007C7C007F7F00000503000000001C22414A
:1029100000000041221C000014083E0814000808B2
:102920003E0808000000503000002010080402009B
:102930000204081020000000000000000000000059
:10294000000000000080E0F8F8F8F0C0000008087F
:102950001838F8F8F8F8F808080000000000000837
:1029600008F8F878180808000808D8F8F8F8F8788F
:102970000808080818F8F8F0F0E00000000088885F
:10298000888888888888F80000000000000000001F
:10299000000000000000C0F03E0F01030F3FFFFFEA
:1029A000FEF8E000000001071FFFFFFFFCF08000C1
:1029B0000000C0F81F0701000000000080F8FFFFC2
:1029C000FF7F2760E0E0F0F8DC1F0F0F0701000039
:1029D000000078444444447850484400000000001B
:1029E000000000008080C0E0F8FEC7818101010185
:1029F00001018187FFFFFFFFFCE0C0808000031F13
:102A00007FFFFFFE7C0F0300000000808080C0F885
:102A1000FFFFFFFFCF80800001071F7FFFFFFCF05B
:102A2000C080800000007C040808102020407D0049
:102A30000000000000000000000000000000080886
:102A4000F8F8F80800000000000000000000000096
:102A5000000000000000000000181818000000002E
:102A60000000000000000000000000000000000066
:102A7000000000000000000000003E22222222226E
:102A800022223E000000000000000000F8FCFE07CB
:102A90000181F1FFFF1F000078FCFE9311190F8FD9
:102AA00046808E9E1F39F9F3E30301E1FFFF1F000B
:102AB0000000F8FCFE070301E1FEFF1F010181FF9A
:102AC000FF7F0602F1FFFF1E0000000000009F9044
:102AD0009090909090909F000000000000000000F7
:102AE00000010101010000010101010000000101DC
:102AF00001010100000001010101010000000000CE
:102B00000101010100000C1D1911191F0F0701001F
:102B100000000101010000000001010101000000AE
:102B2000000010101010101010101F000000A881DD
:102B3000B98188278C930E940E25A1E0B1E08C9387
:102B400000910101003011F00C94A8150C94D215DD
:102B50000D3011F00C94AE150C94D2150A3011F012
:102B60000C94BD15A881B9818C91803011F40C941E
:102B7000BB150C94D4150C94D215009101010F31A2
:102B800018F011F00C94C6150C94D215A1E0B1E028
:102B90008C91A881B9818F930E9401258F918D938B
:102BA00088278C930C949B15089584E690E00E94EE
:102BB00084250E940E25A1E0B1E08C9300910101D3
:102BC000003011F00C94D91508950E940825A2E058
:102BD000B1E08C9300910201013011F00C94521776
:102BE000A2E3B2E0BA93AA930E9497152296E2E379
:102BF000F2E004E0A3E0B1E00E945227A3E0B1E0DC
:102C0000EEE4F1E50E948B2711F00C944C17A2E33F
:102C1000B2E00E948527EA2FFB2F3397F0400FEF99
:102C2000A3E1B1E00E945227E3E1F1E001E0A6E177
:102C3000B1E00E945227A6E1B1E0EAE2F1E50E948C
:102C40008B2711F00C943116A2E3B2E00E94852785
:102C5000EA2FFB2F3297F0400FEFA3E1B1E00E9483
:102C60005227E1E0F0E00E944D25AFE9B0E088276F
:102C70008C93E4E5F1E50E943F25A3E1B1E00E94D9
:102C800039250E9446258AE090E00E948425A2E32F
:102C9000B2E0BA93AA930E94971522968AE090E038
:102CA0000E948425A2E3B2E0BA93AA930E949715EA
:102CB000229686E1E2E3F2E00CE00A93AFE9B0E0AD
:102CC0000E944B27E2E3F2E0A8E1B1E00E94462730
:102CD0008AE090E00E948425A2E3B2E0BA93AA932E
:102CE0000E9497152296E2E3F2E0A8E1B1E00E948B
:102CF0004627E8E1F1E00EE0A8E1B1E00E945227AA
:102D0000DA9884E690E00E948425DA9A82E390E0E3
:102D10000E948425A7E7B2E08C918F5F8C9300918D
:102D200077020A3011F00C94801680E080937702CD
:102D30005A924A9280E0A42DB52D8C9381E00E9496
:102D4000F6245A924A9282E0A42DB52D8C9381E00C
:102D50000E94F6240E94BE09249682E00E94F2247A
:102D60005A924A92A42DB52DEEE5F1E50E949925DF
:102D70008FE00E94F6240E946F0A22968FE00E9444
:102D8000F2245A924A9280E0A42DB52D8C9381E0D2
:102D90000E94F6245A924A9282E0A42DB52D8C937B
:102DA00081E00E94F6240E94BE09249682E00E94DF
:102DB000F2245A924A92EFE9F0E0A42DB52D0E9438
:102DC00046278CE00E94F6240E946F0A22968CE02F
:102DD0000E94F2245A924A9280E0A42DB52D8C9341
:102DE00081E00E94F6245A924A9283E0A42DB52DE8
:102DF0008C9381E00E94F6240E94BE09249682E012
:102E00000E94F2245A924A92A42DB52DEEE5F1E5E6
:102E10000E9499258FE00E94F6240E946F0A229654
:102E20008FE00E94F2245A924A9280E0A42DB52DA0
:102E30008C9381E00E94F6245A924A9283E0A42D5A
:102E4000B52D8C9381E00E94F6240E94BE09249641
:102E500082E00E94F2245A924A92E8E1F1E0A42D25
:102E6000B52D0E94462789E70E94F6240E946F0A2A
:102E7000229689E70E94F224E8EEFFE40E943F25B3
:102E800082E20E944925E2EFFFE40E943F2582E2B0
:102E90000E9449250E94462584E690E00E948425F0
:102EA0000E94D5150895A8E1B1E0E0E2F0E50E94A6
:102EB0008B2711F00C949517969880917A028F7752
:102EC00080937A02ABE7B2E0EEE6F1E50E94992545
:102ED000A8E1B1E088278C935A924A9280E0A42D11
:102EE000B52D8C9381E00E94F6245A924A9283E099
:102EF000A42DB52D8C9381E00E94F6240E94BE097A
:102F0000249682E00E94F2245A924A92A42DB52D72
:102F1000E2E7F1E50E9499258FE00E94F6240E94E5
:102F20006F0A22968FE00E94F224A8E1B1E0E2E26B
:102F3000F0E50E948B2711F00C94D717969A809198
:102F40007A02806880937A02ABE7B2E0E2E8F1E5CA
:102F50000E949925A8E1B1E088278C935A924A9261
:102F600080E0A42DB52D8C9381E00E94F6245A9226
:102F70004A9283E0A42DB52D8C9381E00E94F62423
:102F80000E94BE09249682E00E94F2245A924A923C
:102F9000A42DB52DE6E8F1E50E9499258FE00E9469
:102FA000F6240E946F0A22968FE00E94F224A8E184
:102FB000B1E0E4E2F0E50E948B2711F00C943C189C
:102FC0000E94B41FA8E1B1E088278C93AFE9B0E07C
:102FD00088278C935A924A9280E0A42DB52D8C9329
:102FE00081E00E94F6245A924A9282E0A42DB52DE7
:102FF0008C9381E00E94F6240E94BE09249682E010
:103000000E94F2245A924A92A42DB52DEEE5F1E5E4
:103010000E9499258FE00E94F6240E946F0A229652
:103020008FE00E94F2245A924A9280E0A42DB52D9E
:103030008C9381E00E94F6245A924A9283E0A42D58
:10304000B52D8C9381E00E94F6240E94BE0924963F
:1030500082E00E94F2245A924A92A42DB52DEEE508
:10306000F1E50E9499258FE00E94F6240E946F0AE4
:1030700022968FE00E94F224A8E1B1E0E6E2F0E5BA
:103080000E948B2711F00C94A1180E947120A8E1D6
:10309000B1E088278C93AFE9B0E088278C935A92EF
:1030A0004A9280E0A42DB52D8C9381E00E94F624F5
:1030B0005A924A9282E0A42DB52D8C9381E00E9411
:1030C000F6240E94BE09249682E00E94F2245A92BD
:1030D0004A92A42DB52DEEE5F1E50E9499258FE0E9
:1030E0000E94F6240E946F0A22968FE00E94F2242A
:1030F0005A924A9280E0A42DB52D8C9381E00E94D3
:10310000F6245A924A9283E0A42DB52D8C9381E047
:103110000E94F6240E94BE09249682E00E94F224B6
:103120005A924A92A42DB52DEEE5F1E50E9499251B
:103130008FE00E94F6240E946F0A22968FE00E9480
:10314000F224A8E1B1E0E8E2F0E50E948B2711F05B
:103150000C94BE180E94F91AE6E8F2E0A1E9B1E089
:103160000E944627E0E9F2E0A1E9B1E00E940125D2
:103170000E9446270E94B71A0E94D515A8E1B1E027
:10318000EAE2F0E50E948B2711F00C94D0188091B0
:103190007A028F7B80937A02A8E1B1E088278C9332
:1031A000A8E1B1E0ECE2F0E50E948B2711F00C946D
:1031B000E21880917A02806480937A02A8E1B1E0FB
:1031C00088278C93A8E1B1E0EEE2F0E50E948B271E
:1031D00011F00C94F518E6E9F1E50E943F250E94F4
:1031E0004625A8E1B1E088278C93A8E1B1E0E0E3AF
:1031F000F0E50E948B2711F00C940819EEE9F1E537
:103200000E943F250E944625A8E1B1E088278C93C3
:10321000A8E1B1E0E6EAF1E50E948B2781E009F040
:1032200080E08F93A8E1B1E0ECEAF1E50E948B2702
:1032300081E009F080E09F91892B8F93A8E1B1E0B4
:10324000E2EBF1E50E948B2781E009F080E09F919D
:10325000892B882311F40C94FF19A1E9B1E0E8EB64
:10326000F1E50E9499258AE0A1E9B1E08F930E94DF
:1032700001258F918D9388278C93A1E9B1E00E945D
:103280000125E8ECF1E50E9499258AE0A1E9B1E089
:103290008F930E9401258F918D9388278C93A1E9AC
:1032A000B1E00E940125E4EDF1E50E9499258AE054
:1032B000A1E9B1E08F930E9401258F918D9388271A
:1032C0008C93A1E9B1E00E940125E0EEF1E50E94B6
:1032D00099258AE0A1E9B1E08F930E9401258F91A1
:1032E0008D9388278C93A1E9B1E00E940125E0EF3E
:1032F000F1E50E9499258AE0A1E9B1E08F930E944F
:1033000001258F918D9388278C93A1E9B1E00E94CC
:103310000125EAEFF1E50E9499258AE0A1E9B1E0F3
:103320008F930E9401258F918D9388278C93A1E91B
:10333000B1E00E940125EAE0F2E50E9499258AE0C9
:10334000A1E9B1E08F930E9401258F918D93882789
:103350008C93A1E9B1E00E940125EEE1F2E50E9423
:1033600099258AE0A1E9B1E08F930E9401258F9110
:103370008D9388278C93A1E9B1E00E940125E2E3B7
:10338000F2E50E9499258AE0A1E9B1E08F930E94BD
:1033900001258F918D9388278C93A1E9B1E00E943C
:1033A0000125E8E4F2E50E9499258AE0A1E9B1E06F
:1033B0008F930E9401258F918D9388278C93A1E98B
:1033C000B1E00E940125ECE5F2E50E9499258AE032
:1033D000A1E9B1E08F930E9401258F918D938827F9
:1033E0008C93A1E9B1E00E940125E4E6F2E50E9498
:1033F00099250E94B71AA8E1B1E088278C93A8E12B
:10340000B1E0E0E8F2E50E948B2711F00C94311A4C
:10341000EFE9F0E0ADEDB2E00E944627E0E0F0E039
:10342000ADEDB2E07BE70E946027A1E9B1E0ECE8F6
:10343000F2E50E949925EDEDF2E0A1E9B1E00E94EC
:1034400001250E944627A1E9B1E00E940125E6E995
:10345000F2E50E9499250E94B71AA8E1B1E08827F9
:103460008C93A8E1B1E0E0E4F1E50E948B2711F034
:103470000C94B61AA1E9B1E0EAE9F2E50E949925B7
:103480008AE0A1E9B1E08F930E9401258F918D938D
:1034900088278C93A1E9B1E00E940125E2EAF2E5D8
:1034A0000E949925E6E8F2E0A1E9B1E00E94012539
:1034B0000E944627E0E9F2E0A1E9B1E00E9401257F
:1034C0000E9446278AE0A1E9B1E08F930E9401257E
:1034D0008F918D9388278C93A1E9B1E00E940125FB
:1034E000E8EAF2E50E949925EBE7F2E0A1E9B1E014
:1034F0000E9401250E9446278AE0A1E9B1E08F934E
:103500000E9401258F918D9388278C93A1E9B1E0CA
:103510000E940125EEEAF2E50E949925EFE7F2E02C
:10352000A1E9B1E00E9401250E9446278AE0A1E9B5
:10353000B1E08F930E9401258F918D9388278C9302
:10354000A1E9B1E00E940125EAEBF2E50E9499258C
:10355000E1E8F2E0A1E9B1E00E9401250E944627DE
:103560000E94B71AA8E1B1E088278C930895E2ED94
:10357000F2E50E943F2582E20E944925ADEDB2E0CE
:103580000E94392582E20E9449250E94462588EC46
:1035900090E00E948425A1E9B1E00E9439258AE1EA
:1035A0000E9449250E9446258AE10E944925E1E0C2
:1035B000F0E00E944D258DE00E9449250E9446259D
:1035C000DA9884E690E00E948425DA9A82E390E01B
:1035D0000E948425A7E7B2E08C918F5F8C930091C5
:1035E00077020A3011F00C94E01A80E080937702A1
:1035F000089583E0E0E30E94FA25002762FA0EF4C2
:1036000001E041E0041711F00C943B1B8FEF809315
:103610008502A6E8B2E0ECEDF2E50E9499255A9207
:103620004A9280E0A42DB52D8C9381E00E94F6246F
:103630005A924A9281E0A42DB52D8C9381E00E948C
:10364000F6240E94BE09249682E00E94F2245A9237
:103650004A92E6E8F2E0A42DB52D0E94462786E0C6
:103660000E94F6240E946F0A229686E00E94F224AD
:1036700008950C94E51B6CEC83E0E0E3BB27A6E126
:1036800021E02A930E942D2664E483E0E0E3BB2737
:10369000A6E121E02A930E942D268EEE92E00E9460
:1036A000842583E0E0E30E94FA256CEC83E0E0E30C
:1036B000BB27A6E121E02A930E942D266EEB83E032
:1036C000E0E3BB27A6E121E02A930E942D26BB2739
:1036D000A6E183E0E0E321E02A930E945726ACE8CC
:1036E000B2E05C93BB27A6E183E0E0E321E02A930C
:1036F0000E945726ADE8B2E05C9300918D02083F2E
:1037000018F011F00C94861B0C949C1B0FEF409149
:103710008C02041BACE8B2E00C930FEF40918D02D9
:10372000041BADE8B2E00C93A6E8B2E0E6E1F1E5F7
:103730000E9499250C94A21BA6E8B2E0ECE3F1E507
:103740000E94992500918C0240E10E947527AEE805
:10375000B2E00C9300918D0240E1049FAFE8B2E02B
:103760000C9200918E0240918F02040FA5E8B2E006
:103770000C93A6E8B2E0E6E1F1E50E948B2711F098
:103780000C94C91B00918E0241E0040FA5E8B2E041
:103790000C93A6E8B2E0ECE3F1E50E948B2781E010
:1037A00009F080E08F9300918502003081E009F0FC
:1037B00080E09F918923882311F40C94E51BA6E8EF
:1037C000B2E0E4E1F1E50E949925A0E9B2E0E5E884
:1037D000F2E00E94CA26E0E9F2E0ACE7B7E00E941E
:1037E0004627ECE7F7E0A0E9B2E01127222700E046
:1037F00033270E94AD255A924A9280E0A42DB52D20
:103800008C9381E00E94F6245A924A9281E0A42D82
:10381000B52D8C9381E00E94F6240E94BE09249667
:1038200082E00E94F2245A924A92A42DB52DEEE530
:10383000F1E50E9499258FE00E94F6240E946F0A0C
:1038400022968FE00E94F2245A924A9280E0A42DA0
:10385000B52D8C9381E00E94F6245A924A9281E021
:10386000A42DB52D8C9381E00E94F6240E94BE0900
:10387000249682E00E94F2245A924A92E6E8F2E00C
:10388000A42DB52D0E94462786E00E94F6240E94B2
:103890006F0A229686E00E94F2245A924A9281E0B0
:1038A000A42DB52D8C9381E00E94F6245A924A9261
:1038B00081E0A42DB52D8C9381E00E94F6240E9416
:1038C000BE09249682E00E94F2245A924A92E0E9CC
:1038D000F2E0A42DB52D0E94462785E00E94F62433
:1038E0000E946F0A229685E00E94F2245A924A9220
:1038F00083E0A42DB52D8C9381E00E94F6245A928A
:103900004A9281E0A42DB52D8C9381E00E94F6248B
:103910000E94BE09249682E00E94F2245A924A92A2
:10392000A42DB52DE2EEF2E50E94992583E00E94D8
:10393000F6240E946F0A229683E00E94F2240895E2
:10394000E6EEF2E50E943F250E94462584EF91E0D5
:103950000E948425A2E3B2E0BA93AA930E9497152D
:10396000229684E690E00E948425A2E3B2E0BA9316
:10397000AA930E9497152296E2E3F2E0AEE9B2E044
:103980000E9446278CE0EEE9F2E009E00A93AEE9F6
:10399000B2E00E944B275A924A9280E0A42DB52DA6
:1039A0008C9381E00E94F6245A924A9280E0A42DE2
:1039B000B52D8C9381E00E94F6240E94BE092496C6
:1039C00082E00E94F2245A924A92A42DB52DE0EF93
:1039D000F2E50E9499258CE00E94F6240E946F0A6D
:1039E00022968CE00E94F2245A924A9280E0A42D02
:1039F000B52D8C9381E00E94F6245A924A9280E081
:103A0000A42DB52D8C9381E00E94F6240E94BE095E
:103A1000249682E00E94F2245A924A92EEE9F2E061
:103A2000A42DB52D0E94462785E10E94F6240E9410
:103A30006F0A229685E10E94F2240E94D51508950E
:103A40005A924A928BE0A42DB52D8C9381E00E946E
:103A5000F6245A924A9280E0A42DB52D8C9381E0F1
:103A60000E94F6240E94BE09249682E00E94F2245D
:103A70005A924A92A42DB52DEEE3F1E50E949925C4
:103A800082E00E94F6240E946F0A229682E00E9441
:103A9000F224ECEFF2E50E943F250E9446258CE2DD
:103AA00091E00E948425A2E3B2E0BA93AA930E9417
:103AB0009715229684E690E00E948425A2E3B2E066
:103AC000BA93AA930E9497152296E2E3F2E0A6E940
:103AD000B2E00E94462787E0E6E9F2E002E00A93BE
:103AE000A6E9B2E00E944B27A6E9B2E00E941427A3
:103AF000ADE9B2E00C935A924A928CE0A42DB52D18
:103B00008C9381E00E94F6245A924A9280E0A42D80
:103B1000B52D8C9381E00E94F6240E94BE09249664
:103B200082E00E94F2245A924A92A42DB52DE4E03C
:103B3000F3E50E94992583E00E94F6240E946F0A13
:103B4000229683E00E94F22400919D02003080E0E2
:103B500010F009F081E08F9300919D02043081E024
:103B600008F080E09F918923882311F40C94E31DD1
:103B70005A924A928CE0A42DB52D8C9381E00E943C
:103B8000F6245A924A9280E0A42DB52D8C9381E0C0
:103B90000E94F6240E94BE09249682E00E94F2242C
:103BA0005A924A92A42DB52DE8E0F3E50E9499259A
:103BB00083E00E94F6240E946F0A229683E00E940E
:103BC000F2240C94DC1E00919D02043080E010F081
:103BD00009F081E08F9300919D02093081E008F0A7
:103BE00080E09F918923882311F40C94221E5A921D
:103BF0004A928CE0A42DB52D8C9381E00E94F6248E
:103C00005A924A9280E0A42DB52D8C9381E00E94B7
:103C1000F6240E94BE09249682E00E94F2245A9261
:103C20004A92A42DB52DECE0F3E50E94992583E09E
:103C30000E94F6240E946F0A229683E00E94F224DA
:103C40000C94DC1E00919D02093080E010F009F018
:103C500081E08F9300919D020F3081E008F080E0B9
:103C60009F918923882311F40C94611E5A924A92E1
:103C70008CE0A42DB52D8C9381E00E94F6245A92FD
:103C80004A9280E0A42DB52D8C9381E00E94F62409
:103C90000E94BE09249682E00E94F2245A924A921F
:103CA000A42DB52DE0E1F3E50E94992583E00E9463
:103CB000F6240E946F0A229683E00E94F2240C945C
:103CC000DC1E00919D020F3080E010F009F081E0D1
:103CD0008F9300919D02003281E008F080E09F9177
:103CE0008923882311F40C94A01E5A924A928CE0E6
:103CF000A42DB52D8C9381E00E94F6245A924A920D
:103D000080E0A42DB52D8C9381E00E94F6240E94C2
:103D1000BE09249682E00E94F2245A924A92A42D6F
:103D2000B52DE4E1F3E50E94992583E00E94F62495
:103D30000E946F0A229683E00E94F2240C94DC1EFB
:103D400000919D02003081E009F080E08F930091A6
:103D50009D02033681E009F080E09F91892B882342
:103D600011F40C94DC1E5A924A928CE0A42DB52DCD
:103D70008C9381E00E94F6245A924A9280E0A42D0E
:103D8000B52D8C9381E00E94F6240E94BE092496F2
:103D900082E00E94F2245A924A92A42DB52DECE2C0
:103DA000F1E50E94992582E00E94F6240E946F0AA4
:103DB000229682E00E94F2240E94D5150895E8E13F
:103DC000F3E50E943F250E94462580E991E00E948C
:103DD0008425A2E3B2E0BA93AA930E949715229693
:103DE00080E991E00E948425A2E3B2E0BA93AA930D
:103DF0000E949715229689E0E2E3F2E008E00A9338
:103E0000A3EBB2E00E944B275A924A9280E0A42D85
:103E1000B52D8C9381E00E94F6245A924A9285E057
:103E2000A42DB52D8C9381E00E94F6240E94BE093A
:103E3000249682E00E94F2245A924A92A42DB52D33
:103E4000EEE5F1E50E9499258FE00E94F6240E949C
:103E50006F0A22968FE00E94F2245A924A9280E0E2
:103E6000A42DB52D8C9381E00E94F6245A924A929B
:103E700085E0A42DB52D8C9381E00E94F6240E944C
:103E8000BE09249682E00E94F2245A924A92E3EB01
:103E9000F2E0A42DB52D0E94462785E10E94F6246C
:103EA0000E946F0A229685E10E94F22482E1E2E3F9
:103EB000F2E005E00A93A8ECB2E00E944B275A9288
:103EC0004A9280E0A42DB52D8C9381E00E94F624C7
:103ED0005A924A9284E0A42DB52D8C9381E00E94E1
:103EE000F6240E94BE09249682E00E94F2245A928F
:103EF0004A92A42DB52DEEE5F1E50E9499258FE0BB
:103F00000E94F6240E946F0A22968FE00E94F224FB
:103F10005A924A9280E0A42DB52D8C9381E00E94A4
:103F2000F6245A924A9284E0A42DB52D8C9381E018
:103F30000E94F6240E94BE09249682E00E94F22488
:103F40005A924A92E8ECF2E0A42DB52D0E94462741
:103F500085E10E94F6240E946F0A229685E10E9464
:103F6000F2240E94D5150895E2E2F3E50E943F2570
:103F7000ADEDB2E00E943925E6E4F1E50E943F256F
:103F80000E94462584E690E00E9484255A924A9237
:103F900080E0A42DB52D8C9381E00E94F6245A92E6
:103FA0004A9282E0A42DB52D8C9381E00E94F624E4
:103FB0000E94BE09249682E00E94F2245A924A92FC
:103FC000A42DB52DEEE5F1E50E9499258FE00E9424
:103FD000F6240E946F0A22968FE00E94F2245A92E1
:103FE0004A9280E0A42DB52D8C9381E00E94F624A6
:103FF0005A924A9282E0A42DB52D8C9381E00E94C2
:10400000F6240E94BE09249682E00E94F2245A926D
:104010004A92A42DB52DE6E2F3E50E9499258AE0A7
:104020000E94F6240E946F0A22968AE00E94F224DF
:104030005A924A9280E0A42DB52D8C9381E00E9483
:10404000F6245A924A9283E0A42DB52D8C9381E0F8
:104050000E94F6240E94BE09249682E00E94F22467
:104060005A924A92A42DB52DEEE5F1E50E949925CC
:104070008FE00E94F6240E946F0A22968FE00E9431
:10408000F2245A924A9280E0A42DB52D8C9381E0BF
:104090000E94F6245A924A9283E0A42DB52D8C9367
:1040A00081E00E94F6240E94BE09249682E00E94CC
:1040B000F2245A924A92EDEDF2E0A42DB52D0E9421
:1040C00046278DE00E94F6240E946F0A22968DE01A
:1040D0000E94F224E4E1F0E00E944D250E94D515F3
:1040E00008955A924A9280E0A42DB52D8C9381E0D8
:1040F0000E94F6245A924A9282E0A42DB52D8C9308
:1041000081E00E94F6240E94BE09249682E00E946B
:10411000F2245A924A92A42DB52DEEE5F1E50E94C3
:1041200099258FE00E94F6240E946F0A22968FE064
:104130000E94F2245A924A9280E0A42DB52D8C93CD
:1041400081E00E94F6245A924A9282E0A42DB52D75
:104150008C9381E00E94F6240E94BE09249682E09E
:104160000E94F2245A924A92A42DB52DE0E3F3E581
:104170000E9499258FE00E94F6240E946F0A2296E1
:104180008FE00E94F2245A924A9280E0A42DB52D2D
:104190008C9381E00E94F6245A924A9283E0A42DE7
:1041A000B52D8C9381E00E94F6240E94BE092496CE
:1041B00082E00E94F2245A924A92A42DB52DEEE597
:1041C000F1E50E9499258FE00E94F6240E946F0A73
:1041D00022968FE00E94F224E0E4F3E50E943F255E
:1041E0000E944625E1E0F0E00E944D25A2E3B2E006
:1041F000BA93AA930E9497152296A2E3B2E0BA93CB
:10420000AA930E9497152296A2E3B2E0BA93AA93CA
:104210000E9497152296E2E3F2E0A1E9B1E00E9444
:1042200046270E94B71A0E94D51508955A924A92BD
:1042300080E0A42DB52D8C9381E00E94F6245A9243
:104240004A9283E0A42DB52D8C9381E00E94F62440
:104250000E94BE09249682E00E94F2245A924A9259
:10426000A42DB52DEEE5F1E50E9499258FE00E9481
:10427000F6240E946F0A22968FE00E94F224002703
:10428000AAE7B2E08C9187FB0EF401E040E004174E
:1042900011F00C947C215A924A9280E0A42DB52D05
:1042A0008C9381E00E94F6245A924A9283E0A42DD6
:1042B000B52D8C9381E00E94F6240E94BE092496BD
:1042C00082E00E94F2245A924A92A42DB52DE2E790
:1042D000F1E50E9499258FE00E94F6240E946F0A62
:1042E00022968FE00E94F224ABE7B2E0EEE6F1E521
:1042F0000E9499250C94AB215A924A9280E0A42DF9
:10430000B52D8C9381E00E94F6245A924A9283E064
:10431000A42DB52D8C9381E00E94F6240E94BE0945
:10432000249682E00E94F2245A924A92A42DB52D3E
:10433000E6E8F1E50E9499258FE00E94F6240E94AC
:104340006F0A22968FE00E94F224ABE7B2E0E2E827
:10435000F1E50E9499250027A0E3B0E08C9184FB51
:104360000EF401E040E0041711F00C940B225A9275
:104370004A9280E0A42DB52D8C9381E00E94F62412
:104380005A924A9282E0A42DB52D8C9381E00E942E
:10439000F6240E94BE09249682E00E94F2245A92DA
:1043A0004A92A42DB52DEEE5F1E50E9499258FE006
:1043B0000E94F6240E946F0A22968FE00E94F22447
:1043C0005A924A9280E0A42DB52D8C9381E00E94F0
:1043D000F6245A924A9282E0A42DB52D8C9381E066
:1043E0000E94F6240E94BE09249682E00E94F224D4
:1043F0005A924A92A42DB52DEAE4F3E50E9499253C
:104400008FE00E94F6240E946F0A22968FE00E949D
:10441000F2240C9471225A924A9280E0A42DB52D78
:104420008C9381E00E94F6245A924A9282E0A42D55
:10443000B52D8C9381E00E94F6240E94BE0924963B
:1044400082E00E94F2245A924A92A42DB52DEEE504
:10445000F1E50E9499258FE00E94F6240E946F0AE0
:1044600022968FE00E94F2245A924A9280E0A42D74
:10447000B52D8C9381E00E94F6245A924A9282E0F4
:10448000A42DB52D8C9381E00E94F6240E94BE09D4
:10449000249682E00E94F2245A924A92A42DB52DCD
:1044A000EAE5F3E50E9499258CE00E94F6240E943B
:1044B0006F0A22968CE00E94F224E2E0F0E00E9473
:1044C0004D250027A0E3B0E08C9184FB0EF401E0C1
:1044D00041E0041711F00C9471220C947D000C94AF
:1044E00071220E94D5158AE090E00E9484250895EB
:1044F0000027A0E3B0E08C9187FB0EF401E041E0DF
:10450000041711F00C9424235A924A9286E0A42DA9
:10451000B52D8C9381E00E94F6245A924A9281E054
:10452000A42DB52D8C9381E00E94F6240E94BE0933
:10453000249682E00E94F2245A924A92A42DB52D2C
:10454000E6E6F3E50E94992589E00E94F6240E94A0
:104550006F0A229689E00E94F224AFE7B2E0E2E21D
:10456000F0E50E949925E1E0F0E00E944D2500274A
:10457000AAE7B2E08C9186FB0EF401E040E004175C
:1045800011F00C942223A1E9B1E0E0E7F3E50E94E9
:1045900099255A924A9280E0A42DB52D8C9381E002
:1045A0000E94F6245A924A9281E0A42DB52D8C9354
:1045B00081E00E94F6240E94BE09249682E00E94B7
:1045C000F2245A924A92A42DB52DEEE5F1E50E940F
:1045D00099258FE00E94F6240E946F0A22968FE0B0
:1045E0000E94F2245A924A9280E0A42DB52D8C9319
:1045F00081E00E94F6245A924A9281E0A42DB52DC2
:104600008C9381E00E94F6240E94BE09249682E0E9
:104610000E94F2245A924A92A42DB52DE8E7F3E5C0
:104620000E9499258FE00E94F6240E946F0A22962C
:104630008FE00E94F2240E94B71A80917A0280646F
:1046400080937A020C9453235A924A9286E0A42DC6
:10465000B52D8C9381E00E94F6245A924A9281E013
:10466000A42DB52D8C9381E00E94F6240E94BE09F2
:10467000249682E00E94F2245A924A92A42DB52DEB
:10468000E8E8F3E50E94992589E00E94F6240E945B
:104690006F0A229689E00E94F224AFE7B2E0E0E2DE
:1046A000F0E50E9499250027AAE7B2E08C9186FBED
:1046B0000EF401E040E0041711F00C9490235A929C
:1046C0004A928DE0A42DB52D8C9381E00E94F624B2
:1046D0005A924A9281E0A42DB52D8C9381E00E94DC
:1046E000F6240E94BE09249682E00E94F2245A9287
:1046F0004A92A42DB52DE4E1F1E50E94992582E0CE
:104700000E94F6240E946F0A229682E00E94F22400
:10471000A1E8B2E0E2E9F3E50E9499250C94BF23F9
:104720005A924A928DE0A42DB52D8C9381E00E947F
:10473000F6245A924A9281E0A42DB52D8C9381E003
:104740000E94F6240E94BE09249682E00E94F22470
:104750005A924A92A42DB52DE0E3F1E50E949925E5
:1047600082E00E94F6240E946F0A229682E00E9454
:10477000F224A1E8B2E0E6E9F3E50E9499250E945F
:10478000D5158AE090E00E9484250895EAE9F3E5D2
:104790000E943F250E9446258AE090E00E948425E1
:1047A000A2E3B2E0BA93AA930E94971522968AE0F8
:1047B00090E00E948425A2E3B2E0BA93AA930E94FB
:1047C0009715229686E1E2E3F2E00CE00A93AFE966
:1047D000B0E00E944B27E2E3F2E0A8E1B1E00E94E2
:1047E0004627E8E1F1E004E0A8E1B1E00E945227A9
:1047F000A8E1B1E0E4EAF3E50E948B2711F00C9404
:10480000E5248AE090E00E948425A2E3B2E0BA9316
:10481000AA930E9497152296E2E3F2E0A8E1B1E0A4
:104820000E944627E8E1F1E00EE0A8E1B1E00E9435
:104830005227DA9884E690E00E948425DA9A82E38F
:1048400090E00E948425A7E7B2E08C918F5F8C9363
:10485000009177020A3011F00C94192480E08093C3
:1048600077025A924A9280E0A42DB52D8C9381E074
:104870000E94F6245A924A9282E0A42DB52D8C9380
:1048800081E00E94F6240E94BE09249682E00E94E4
:10489000F2245A924A92A42DB52DEEE5F1E50E943C
:1048A00099258FE00E94F6240E946F0A22968FE0DD
:1048B0000E94F2245A924A9280E0A42DB52D8C9346
:1048C00081E00E94F6245A924A9282E0A42DB52DEE
:1048D0008C9381E00E94F6240E94BE09249682E017
:1048E0000E94F2245A924A92EFE9F0E0A42DB52DED
:1048F0000E9446278CE00E94F6240E946F0A2296AE
:104900008CE00E94F2245A924A9280E0A42DB52DA8
:104910008C9381E00E94F6245A924A9283E0A42D5F
:10492000B52D8C9381E00E94F6240E94BE09249646
:1049300082E00E94F2245A924A92A42DB52DEEE50F
:10494000F1E50E9499258FE00E94F6240E946F0AEB
:1049500022968FE00E94F2245A924A9280E0A42D7F
:10496000B52D8C9381E00E94F6245A924A9283E0FE
:10497000A42DB52D8C9381E00E94F6240E94BE09DF
:10498000249682E00E94F2245A924A92E8E1F1E0F1
:10499000A42DB52D0E94462789E70E94F6240E9487
:1049A0006F0A229689E70E94F224E8EEFFE40E9453
:1049B0003F2582E20E944925E2EFFFE40E943F2565
:1049C00082E20E9449250E94462584E690E00E94EA
:1049D00084250E94D51508958E2E9F2E0895E82DCA
:1049E000F92D0895481A8827580A0895480E8827EF
:1049F000581E0895ED91FC91EF5FFF4FFC93EE93ED
:104A000008958F938D918823E9F711978F910895D9
:104A100080919E00882309F081E0089580919E0096
:104A2000882309F408950F929F93AF93BF937F93C8
:104A300080919E008823E1F3F89480919E008A95EE
:104A400080939E0090919C00A0E6B0E0A90F002406
:104A5000B01D8C9193959C3309F4992790939C00F9
:104A600078947F91BF91AF919F910F900895ACE79B
:104A7000B7E08D91882311F00CD0FBCF08950E94F0
:104A80009F25802D11F005D0FACF08958DE001D03B
:104A90008AE05D9BFECF8CB9089588EE93E034D018
:104AA0003197D9F708953197F1F708950E94662557
:104AB0008D910E946A259A95D9F70E9469250895DB
:104AC000DB98D39ADC98D49AD1980895DB98DC9837
:104AD0000895089508E0880F10F4DC9A02C0DC986D
:104AE0000000DB9A0058005EF0F3DB980058005E8F
:104AF000F0F3C99983950A9571F70895689462F85F
:104B00000895E89462F80895EF93FF93EE27E82B59
:104B1000E92B31F0E0EAFFE03197F1F70197D1F7A7
:104B2000FF91EF9108955A924A92480E8827581E95
:104B300008950E949F250D920020D9F70895C895E9
:104B400031960020089591E0882321F08894991FE0
:104B50008A95E9F7892F909508952E2E3F2E992753
:104B600081918D3209F093958823D1F79A95E22DA2
:104B7000F32D112361F0091718F011F0101B01C07B
:104B8000191B28F021F080E28D931A95E9F78081B6
:104B90008D3219F48D93319604C0222311F08BE2EB
:104BA0008D93091738F031F0091B21F080E38D93C4
:104BB0000A95E9F781918D938823E1F7332351F02A
:104BC000EA2FFB2F319633958E9182933A95E1F738
:104BD0008EE28C9308950181082B018312811923A1
:104BE0001283EF93FF93E4E0F0E00E945325FF91DE
:104BF000EF9108950E947E25FF270E94A325EBDFF9
:104C0000EF93FF93ECE7F7E00E945325FF91EF91BC
:104C1000182B128309230183EF93FF93E4E6F1E05D
:104C20000E945325FF91EF911081182369F4EF93AF
:104C3000FF93ECE7F7E00E945325FF91EF9110817D
:104C4000182311F00E948125EF93FF93ECE7F7E022
:104C50000E945325FF91EF9108950E94A325FF27FD
:104C600029915D9148E0B7DFEF93FF93E4E0F0E036
:104C70000E945325FF91EF91579510F4182B128342
:104C8000EF93FF93ECEEF0E00E945325FF91EF913C
:104C9000182B1283EF93FF93E4E0F0E00E9453257A
:104CA000FF91EF914A95F9F62A95D9F608950E9459
:104CB000A325FF27299148E055278DDF092301838C
:104CC000EF93FF93E4E1F0E00E945325FF91EF9111
:104CD00088941081182309F008945795EF93FF9357
:104CE000E0EBF0E00E945325FF91EF914A9529F700
:104CF0005D932A9501F708957F930F93AF93BF9328
:104D00008F939F938FB78F9380919E000CE3081B26
:104D100021F49CB10E947E2512C000919D00A0E666
:104D2000B0E077279CB1A00FB71F9C938395809329
:104D30009E0003950C3309F4002700939D008F918A
:104D40008FBF9F918F91BF91AF910F917F911895D8
:104D5000040F151F261F371F0895000F111F221F54
:104D6000331F089500951095209530950F5F1F4FC4
:104D70002F4F3F4F0895019110810EC00191119165
:104D8000219130810BC00191108117FF05C03FEFC9
:104D90002FEF04C0008111272227332737FF03C0DC
:104DA000E1DF8DE28D93CF93DF93CF92DF92EF928D
:104DB000AA24BB24CC24DD24EE2440E2CAE0DD2773
:104DC00055E093E38881890F87FD9F7083FD907F75
:104DD000891B89935A95A9F7C0DFAA1CBB1CCC1C60
:104DE000DD1CEE1C4A9551F7E894EFE0FF27829115
:104DF0000ED0EB30E0F71EF068948A2D0CD0882797
:104E00008D93EF90DF90CF90DF91CF910895982F01
:104E1000829501D0892F8F70805D26F0803309F450
:104E2000089568948D93089500271127222733272A
:104E30001DD08A3328F4803318F005D015D0F9CF6F
:104E40000EF490CF089580538F93402F512F622FEF
:104E5000732F83DF82DF7CDF80DF8F919927080F3C
:104E6000191F291F391F08958D910895E894FCDFBB
:104E70008032E9F38B32D9F38930C9F38D3211F4E2
:104E80006894F2CF089588278D93089581918D932A
:104E90008823E1F7089509919191992351F08A951A
:104EA000D9F7319781918D930A9519F08823D1F71D
:104EB0000895E9CFE199FECFEEBBFFBB319608958F
:104EC000F9DF8D917B3729F48DBBE29AE19A882333
:104ED000B9F777270895EEDFE09A8DB38D93882395
:104EE00019F09A95C1F79D930895FF93881BF9E0F7
:104EF000001FFA9511F4FF910895881F841B18F480
:104F0000840F8894F5CF0894F3CF8FEF83959D910C
:104F10009923E1F70895689401C0E894AF93BF9393
:104F20008D9116F0919103C00E949F25902D8917B5
:104F300018F011F48823A1F7BF91AF91089552653D
:104F4000762E3132313132302E64000047534D20FD
:104F500053494D39303044002D2D2D2D2D2D2D2D23
:104F60002D2D2D2D2D2D000041565270726F6A652A
:104F700063742E727500C2EAEBFEF7E5EDE8E520FA
:104F8000202020200000DAFAFAFAFAFAFAFAFAFAFD
:104F9000FAFAFADB0000D900D800D600D700D0E535
:104FA000E3E8F1F2F0E0F6E8FF2020200000DA006C
:104FB000CEF7E8F1F2EAE020E1F3F4E5F0E00000FA
:104FC00041540000C2E5F0E8F4E8EAE0F6E8FF202A
:104FD000415400004F4B0000D3E4E0EBE5EDE8E581
:104FE00020534D532020000041542B434D47444152
:104FF0003D0044454C20414C4C00C90053494D39BB
:1050000030304420E3EEF2EEE221000041542B4325
:105010004D47463D310041542B434C49503D3100F2
:1050200030003100320033003400350036003700E4
:10503000380039004100420043004400450046006A
:105040004700480049004A004B004C004D004E000C
:105050004F005000510052005300540055005600BC
:105060005700580059005A00610062006300640054
:10507000650066006700680069006A006B006C00EC
:105080006D006E006F00700071007200730074009C
:10509000750076007700780079007A00C000E000A3
:1050A000C100E100C200E200C300E300C400E4006C
:1050B000C500E500A800B800C600E600C700E7008C
:1050C000C800E800E900CA00EA00CB00EB00CC0011
:1050D000EC00CD00ED00CE00EE00CF00EF00D000E0
:1050E000F000D100F100D200F200D300F300D500AF
:1050F000F500F700F600D400F400F800F900DC0039
:10510000FC00FA00DB00FB00DD00FD00DE00FE001D
:10511000DF00FF0020002D002E003A003E00B0000E
:105120004000260027003C002A002C0024003D00FF
:105130002100BD00230028005B0025002B005E003D
:105140003F005D0029003B002F005C005F002B4307
:105150004D54000041542B434D47523D0000202048
:1051600020202020202020202020202000004F660A
:1051700066004C6F6164204F46462020202020208E
:1051800000004F4E00004C6F6164204F4E202020E5
:10519000202020200000415453303D300000415475
:1051A00053303D32000068656C70000048656C70DB
:1051B000000048454C50000053494D3930304420E0
:1051C00068656C7065720000303A204F6666206C2E
:1051D0006F616400313A204F6E206C6F6164000093
:1051E000323A20506572657A766F6E6974270000D6
:1051F000333A2042616C616E7300343A2054656D1D
:1052000070657261747572650000353A20456E6193
:10521000626C652073656E6420534D530000363A0E
:105220002044697361626C652073656E6420534D20
:105230005300373A204176746F706F646E796174F1
:105240006965204F66660000383A204176746F70B9
:105250006F646E7961746965204F6E003F3A204932
:105260006E666F0046697273746E756D6265723A30
:10527000204368616E6765206E756D62657200001F
:1052800046697273746E756D626572004E756D62FB
:1052900065723A200000204F4B0053494D393030A1
:1052A000440054656D703A004C6F61643A00504997
:1052B000522073656E736F723A0053656E642053AB
:1052C0004D532066726F6D2073656E736F72733A03
:1052D000000041542B434D47533D00006572726FEF
:1052E0007200B043000041542B434F50533F000025
:1052F00020202020202020202020200041542B434B
:1053000053510000202000003E2000003C200000FF
:105310003C4000003C26000041542B43434C4B3F93
:10532000000041544400C7E2EEEDE8EC20EDE0005F
:10533000C7E0EFF0EEF120E1E0EBE0EDF1E000009E
:105340004154442A31303023000053494D39303024
:1053500044204F4E20202020000053494D3930304A
:1053600044204F464600C4E0F22E203120200000A9
:10537000416C61726D210000CEF2EFF0E0E2EAE0F4
:1053800020534D5320200000C4E0F22E2030202076
:105390000000596573004E6F000041542B434D4788
:0A53A000523D31002B434D47000041
:00000001FF
